:020000040000FA
:060000000F308A000C2FF6
:08000800F200030E8301F50074
:100010000A08F4008A010408F300831203138C1EFB
:1000200027281A08981C18281A08181218160D28BC
:1000300083160313F600A10AE3302102031D2228D0
:10004000A230A10021088400760880000D287308E2
:10005000840074088A00750E8300F20E720E090087
:100060008301831603132730810000308C00003099
:100070008D00EF30850000308600B0308700003002
:100080009F0083120313003085000030860000308B
:100090008700C0308B00003090008C0197019D01DB
:1000A000203084008001840A6D300402031C522831
:1000B000B5231F24042183160313A230A100A0003E
:1000C0008C168312031307142830A5005C30A60099
:1000D0008F30A7000230A800332143216321031C85
:1000E0006E28A800A81BBE286321031C7428A70043
:1000F0006321031C7828A6006321031C7C28A5002B
:1001000043216321031C8128A0007039A100210C28
:100110003839860020080739820796289A289E28B1
:10012000A228A628AC28B228B8286E28C9302021D9
:100130001B216E28C13020211B216E28D1302021A7
:100140001B216E28D93020211B216E28C930202187
:100150001B2124081B216E28C13020211B212408CB
:100160001B216E28D13020211B2124081B216E2841
:10017000D93020211B2124081B216E2828080F3983
:100180008207D228D328D428D528DC28D628EA28E4
:10019000F0286E286E286E286E286E286E286E282D
:1001A0007D296E28A628AC28B228B82861302021E5
:1001B0001B2124081B216E286321031CDC28A700B7
:1001C0006321031CE028A6006321031CE428A5008A
:1001D00062216E286321031CEA2886001B216E28F9
:1001E0006321031CF028A8006321031CF428A70046
:1001F0006321031CF828A6006321031CFC28A5002A
:100200004321AA301B216E2883120313071683167D
:10021000031307121430990018159816831203134C
:10022000181698170712080007128C1E15291A08AD
:100230000800871A19290C1E1B2999000800C130D3
:100240009F002E211F151F192329831603131E0833
:1002500083120313A4001E08A30008000730A000A7
:10026000A00B3029080007100130AA0055210030EA
:10027000AA0055210030AA005521A730AA00552117
:100280008715871108000430AA0055212808AA0004
:1002900055212708AA0055212608AA00552125081E
:1002A000AA0055218715871108000830A200031005
:1002B000AA0D03180715031C071187148710A20B3A
:1002C000582908000800831603132108200283120E
:1002D0000313031D6D290310080083160313A00ADE
:1002E000E3302002031D7629A230A00020088400FC
:1002F0000008831203130314080002226321031C65
:100300007E29E80060306802031802224F30840022
:100310004E08840768088000CE0A4F08773A031D0C
:1003200098294E08163A031D98292B14FC22002AFE
:100330004F08663A031DA2294E080A3A031DA22956
:100340006523002A4F08783A031DAD294E08163A56
:10035000031DAD292B10FC22002A4F086D3A031D06
:10036000B7294E08013A031DB7295423002A4F0824
:10037000653A031DC1294E080D3A031DC129752395
:10038000002A4F08763A031DCB294E08013A031D77
:10039000CB29B123002A4F08723A031DD5294E08F4
:1003A000023A031DD529BB23002A4F08613A031DD9
:1003B000E0294E08193A031DE0292B10FA22002AE1
:1003C0004F08623A031DEB294E08193A031DEB2929
:1003D0002B14FA22002A4F08733A031DF5294E0800
:1003E000013A031DF529A123002A4F086F3A031D86
:1003F000FF294E08023A031DFF29B423002A7E2953
:1004000002226E288C220800D201D301D401D5012A
:10041000D601D701CE01CF01D001D10108000422BD
:10042000480884000008CE00840A0008CF00840A2F
:100430000008D000840A0008D100840A0008D20015
:100440002830AC000310D20CD10CD00CCF0CCE0C49
:10045000D70CD60CD50CD40CD30C4E308400053000
:10046000AD00801F352A30308002801D392A0330CC
:100470008002840AAD0B312AAC0B222A4808840082
:1004800053088000840A54088000840A55088000BC
:10049000840A56088000840A5708800008002E0845
:1004A000D8002F08D9003008DA003108DB00320804
:1004B000DC002030D6005830C8006030C900CF01C1
:1004C0000310D50CD40CD30CD20C031C802A08309A
:1004D000D000480884000008CE00490884004F0876
:1004E000CF018007031C762A0130CF004E08800719
:1004F000031C7C2A0130CF00C80AC90AD00B692A24
:100500000310D80DD90DDA0DDB0DDC0DDD0DDE0D80
:10051000DF0DD60B5B2A08004E3084008001673067
:1005200004020319952A840A8E2A080050080F39FC
:10053000B800510EF039B70052080F39B704530E06
:10054000F039B60054080F39B604550EF039B5002D
:1005500056080F39B504570EF039B40058080F3952
:10056000B4040800BD01590EF039BC005A080F3917
:10057000BC045B0EF039BB005C080F39BB045D0E98
:10058000F039BA005E080F39BA045F0EF039B900CD
:1005900060080F39B9040800C001C101C201610E31
:1005A000F039BF0062080F39BF04630EF039BE0096
:1005B00064080F39BE040800C401C501C601C701A3
:1005C00065080F39C404660EF039C30067080F3997
:1005D000C30408004308EB004408EC000F30EA00B5
:1005E000EA0BF02AEB0BEE2AEC080319F92AEC03CC
:1005F000EE2A0800DC22FE2AC301C401831603137D
:1006000080309F00831203139622B222CC22343012
:10061000C8000F223930C8000F223E30C8000F2218
:100620004330C8000F228C223508D3003408D20092
:100630003608D4003708D5004F22D323C308031D42
:10064000252BC408031D252B262BEA223908B407C5
:100650003A0803183A0FB5073B0803183B0FB607D3
:100660003C0803183C0FB7078C223508D300340828
:10067000D2003608D4003708D5004F22E0232408E2
:100680001B2123081B21DE2324081B2123081B21F7
:10069000D323BE033E0A0319BF03BE08031D1E2B4E
:1006A000BF08031D1E2B08008316031380309F0014
:1006B00083120313E22324081B2123081B21DE23BA
:1006C00024081B2123081B21080096223430C8006F
:1006D0000F228C223508D3003408D2003608D4000B
:1006E0003708D5004F22D32308005008CB23B2008F
:1006F000B20E5108CB23B2045208CB23B100B10E85
:100700005308CB23B1045408CB23B000B00E5508D6
:10071000CB23B0045608CB23AF00AF0E5708CB2332
:10072000AF045808CB23AE00AE0E5908CB23AE045D
:100730005A08CB23B300B30E5B08CB23B3042C249D
:10074000302802301B2169081B21831603138030D7
:100750009F0083120313DC2324081B2123081B2181
:10076000080077301B210800080086013F30860012
:100770003A24860108005008E900860169188614A9
:10078000E918061569198615E9190616691A8616F3
:10079000E91A06170800CE0041304E023030031827
:1007A00037304E0208006508A6006408A5006608F8
:1007B000A7006708A80043299130E52BA130E52B5D
:1007C0002B18E42B8930E52B81309F00F3231F1574
:1007D0001F19E82B831603131E0883120313A400AA
:1007E0001E08A3000800C830CE00CE0BF52B080071
:1007F000831603178C18FA2B8312031770088D00C9
:1008000071088C00831603178C130C158B1355304D
:100810008D00AA308D008C148B170C1183120313DA
:1008200008008312031770088D00831603178C13BA
:100830000C14831203170C088312031308000630EC
:10084000AC002E3084000030F00011248000840AB7
:10085000F00AAC0B252C08000630AC000030F0008C
:100860002E3084000008F100F823840AF00AAC0B53
:10087000322C08001A30EC007730EB005530EA00DB
:0E088000EA0B402CEB0B402CEC0B402C08003C
:101E00000F308A00022F8A013028000000000000F5
:101E10000F308A000A2F00008316031381018312FA
:101E20000313061C1D2FA227EB27831203178C0810
:101E300083120313031D1B2F032FA501A2273F307D
:101E40008E00FF308C00DF27B927D0273A3A031DD8
:101E5000252FA301A9271F39A2000310A20CA9272F
:101E6000A000A927A1000310A00CA10CA927013AEA
:101E700003198E2F2608003A031D8B2FE030200710
:101E800003188B2F283084002208A400A927800083
:101E9000840AA9278000840AA40B462FA9272308B7
:101EA000031D972F0716283084002208A40020085D
:101EB000031D672FFC3021070318672F2514210805
:101EC000043E831203178D000F308F007D2F251CD9
:101ED000972F0F302002031C732F031D972F003004
:101EE00021020318972F2008831203178F008312F3
:101EF00003132108831203178D0000088C00840A45
:101F000000088E00840ADF2783120313A10F892F94
:101F1000A00AA40B572F2E30D727252F4F30D727B5
:101F20004B30D727A2278E018C01DF27962F453013
:101F3000D7275230D7275230D7274F30D7275230A4
:101F4000D727A12F831203170F308F000B308D007E
:101F50000800D027BF3E031C073E0A3EA600A60E7F
:101F6000D027BF3E031C073E0A3EA6042608A3074F
:101F70000800831203130716831603130712143085
:101F800099001815981683120313181698174830DD
:101F9000D7274630D7274D30D7273930D7270800E5
:101FA0008312031307128C1ED32F1A080800831202
:101FB0000313871AD92F0C1EDB2F990008008316F4
:101FC000031784308C0055308D00AA308D008C149E
:101FD0000000000008001F308F05831603178030B3
:0C1FE0008C000C14000000000800000041
:02400E00723FFF
:0C42000018007100C700BC000A0000009C
:00000001FF
